:020000040800F2
:10000000883E002085020008753300080526000898
:100010000D3300088504000891410008000000002D
:10002000000000000000000000000000A501000822
:10003000DD06000800000000010200080B3900087E
:100040009F0200089F0200089F0200089F0200080C
:100050009F0200089F0200089F0200089F020008FC
:100060009F0200089F0200089F0200089F020008EC
:100070009F0200089F02000895050008A1050008DE
:100080009F0200089F0200089F0200089F020008CC
:100090009F0200089F0200089F0200089F020008BC
:1000A0009F0200089F0200089F0200089F020008AC
:1000B0009F02000800000000000000009F020008EE
:1000C0009F0200089F0200089F0200089F0200088C
:1000D0009F020008554100089F0200089F02000887
:1000E0009F0200089F0200080000000000000000BE
:1000F0000000000000000000000000000000000000
:10010000000000009F020008000000009F0200089D
:100110000000000000000000A93900089F0200084C
:100120009F0200089F0200089F0200089F0200082B
:100130009F02000800000000000000000000000016
:100140009F0200089F0200089F02000800000000B4
:100150009F0200089F0200089F0200089F020008FB
:100160009F0200089F0200089F0200080000000094
:100170009F0200089F02000800000000000000002D
:100180009F0200089F0200089F020008DFF810D0BD
:1001900000F00EF9004800479D450008AFF30080CD
:1001A000883E00202C4B1968086800F05AB880F38C
:1001B0000988BFF36F8F4FF0000080F311887047FC
:1001C0000000000008480068006880F308884FF0CD
:1001D000000080F3148862B661B6BFF34F8FBFF39F
:1001E0006F8F00DF00BF00BF08ED00E0DFF80C00FC
:1001F000016841F470010160704700BF88ED00E0C4
:10020000EFF30980BFF36F8F134B1A681EF0100FC6
:1002100008BF20ED108A20E9F04F106009B44FF0BC
:10022000500080F31188BFF34F8FBFF36F8F05F03D
:10023000DFFB4FF0000080F3118809BC19680868E3
:1002400000F014B81EF0100F08BF00F014B880F3CF
:100250000988BFF36F8F7047B4000020EFF305806B
:10026000704730C8B0E8C04FFFF7A1BF30C8B0E852
:10027000C04FFFF7E7BFB0EC088AB0EC08CAFFF741
:10028000E6BF00000648804706480047FEE7FEE755
:10029000FEE7FEE7FEE7FEE7FEE7FEE7FEE7FEE736
:1002A000993900088D0100082DE9F05F054600200E
:1002B00092469B4688460646814640241BE02846D7
:1002C00041464746224600F063F853465A46C01A54
:1002D000914110D311461846224600F04AF82D1AD3
:1002E00067EB01084F4622460120002100F041F84B
:1002F00017EB00094E41201EA4F10104DFDC484643
:1003000031462A46434600F000B830BCBDE8C09FE5
:1003100040EA01039B0703D009E008C9121F08C087
:10032000042AFAD203E011F8013B00F8013B521E07
:10033000F9D27047D2B201E000F8012B491EFBD27E
:1003400070470022F6E710B513460A4604461946E0
:10035000FFF7F0FF204610BD30B5044600200346ED
:1003600000E05B1C934203D2E05CCD5C401BF8D004
:1003700030BD202A04DB203A00FA02F10020704749
:100380009140C2F1200320FA03F3194390407047D3
:10039000202A04DB203A21FA02F00021704721FADA
:1003A00002F3D040C2F12002914008431946704741
:1003B000064C074D06E0E06840F0010394E80700B2
:1003C00098471034AC42F6D3FFF7E4FE28670008E4
:1003D0004867000830B58C1810F8012B12F00F0395
:1003E00001D110F8013B120906D110F8012B03E0EE
:1003F00010F8015B01F8015B5B1EF9D101E001F827
:10040000013B521EFBD1A142E6D3002030BD0000CB
:100410002DE9F0419AB00646A1F11005684602F0B8
:1004200035FA00244FF4007811E004F5007085429D
:1004300001D9474600E02F1B31193A461048FFF713
:1004400067FF3A460E49684602F0A5FD3C44AC42BF
:10045000EBD3694616A802F0F1F9002216A970192B
:100460008B5C845CA34203D1521C102AF8D301E0B8
:10047000102A03D301201AB0BDE8F0810020FAE76A
:1004800058020020FEE730B5002307E001EB8304AB
:10049000056824684FEA34442C605B1CB3EB520FB0
:1004A000F4D3D20703D0026831F82310118000681A
:1004B000006830BD70B500230CE001EB8304258893
:1004C000A6786DBA2D04E47845EA0625254304682C
:1004D00025605B1CB3EB920FEFD394071BD002F0A7
:1004E0000304012C03D1066811F823503570022C47
:1004F00005D101EB83040568248864BA2C80D243BB
:10050000920708D101EB830103680A8852BA1A8066
:100510000268897811700068006870BD70B54FF48A
:1005200080752A4612491348FFF7F2FE124C2068E4
:100530000088A0F52541A53912D0FF2229460D4893
:10054000FFF7F8FE00F08CF920684BF6BB31A0F8FD
:10055000FC10002120F8EC1F4180416003F060F89E
:100560002068B0F8FC1005A003F060FE002070BD0C
:10057000000001085001002040000020636F6E66FB
:1005800069672D3E496170466C61673A2025782085
:100590000D0A0000014800F069BA0000DC0D0020DF
:1005A000014800F063BA0000940D002030B590F8C7
:1005B000444004F01C050124AC40056C6C600468E8
:1005C00063608368102B036803D099600068C26081
:1005D00030BD9A600068C16030BD00007FB53D4C01
:1005E00082784125A27030F8031F49BA8378090444
:1005F00041EA0321C378194300918188837949BA7C
:10060000090441EA0321C379194301910189837ADD
:1006100049BA090441EA0321C37A19430291818945
:10062000837B49BA090441EA0321C37B194303913F
:10063000017C437C03EB0121837CC07C03EB012123
:1006400000EB0123A361E088E1680D54401C80B2F7
:1006500000250D54401C80B2E080012A01D0062202
:1006600003E0B3F5803F02D902220A5404E001F00E
:10067000EBFFE088E1680D54401CE080E188E06811
:1006800001224554491C89B24554491C89B242543F
:10069000491C89B210224554491CE18069460E4824
:1006A000FFF75AFE50B10C48009901600199416072
:1006B000029981600399C160A560A580A188E08846
:1006C000E2680B0A1354401C80B21154401CE080B5
:1006D0007FBD000054000020580A0020704770B50C
:1006E00000231C4611E011F82350055531F8235022
:1006F0002E0A05196E7051F82360360CAE7051F851
:1007000023605B1C360EEE70241D9442EBD370BD4B
:1007100072B6FEE7144A107F1449012801D003285D
:100720000FD10B6823F400730B600B6843F4006374
:100730000B600B6823F400630B600B6843F40073D9
:100740000B60022801D003280BD1086840F48050C8
:100750000860086820F480500860086840F48060F1
:1007600008600020107770479000002000200240B1
:10077000C107054803D0416941F004014161416965
:1007800041F48031416170470020024008494A69C4
:10079000C0B222F47E7242EAC0004861486940F06B
:1007A00002004861486940F48030486170470000A9
:1007B00000200240054910B54C6944F001044C6129
:1007C0000260BFF36F8F436010BD00000020024045
:1007D000094B10B55C69402244F480245C61EFF35E
:1007E000108372B610C910C0521E12F0FF02F9D168
:1007F00083F3108810BD00000020024070B504464D
:1008000000F012FC0646134D08E0601C06D000F014
:100810000BFC801BA04201D3032070BD2869C003DC
:10082000F3D428690C4908400CD00C494A680243AB
:100830004A60810F01D0A969A961810000D02861B7
:10084000012070BD2869C00701D001202861002067
:1008500070BD000000200240FAC30200900000209A
:1008600004484AF2A55100680180012181700221EB
:10087000C1707047400000200549884202D2A0F1B3
:10088000006002E0024949420844C00A7047000083
:1008900000000408F0B5054600201F2301265B1E5A
:1008A00005D303F01F0706FA07F40C42F7D07AB11C
:1008B000082A09D0102A04D0182A07D1072B05D2FC
:1008C00006E0082B02D203E0102B01D30120F0BD7B
:1008D0000028FCD12B68596129688B6823F0180324
:1008E00013438B60F0BD70B504460020022363778C
:1008F00023689D6845F001059D60236A012B0FD098
:10090000022B11D0032B12D1002304E0256851F8EB
:10091000230028605B1C9342F8D32068006806E03F
:100920002046FFF7C7FD02E02046FFF7ACFD01219E
:10093000617770BD10B5040010D0607F20B9002031
:100940002077204600F030F802206077207938B117
:10095000D4E902122046FFF79DFF48B1012010BDE7
:100960002168104848612068816821F01801816081
:100970006079A0B120692168086120688168626996
:1009800021F060011143816020688168A26921F033
:1009900080011143816001206077002010BD4FF07D
:1009A000FF30E8E7B71DC10408B500680649884272
:1009B00008D10648816C41F480518164806C00F458
:1009C0008050009008BD000000300240001002403E
:1009D00010B590F825100022022905D00421C1632A
:1009E00080F82420012010BD01680B6823F00E035D
:1009F0000B6001680B6823F001030B6090F8441052
:100A0000012401F01C0304FA03F1036C596080F81F
:100A1000254080F82420104610BD10B590F8251010
:100A20000024022903D00421C16301241AE00168D3
:100A30000A6822F00E020A6001680A6822F00102C8
:100A40000A6090F84410012301F01C0203FA02F13D
:100A5000026C516080F82530002180F82410816BF1
:100A600001B18847204610BDC06B7047F0B4016CDF
:100A70000B6801680A6890F84440042504F01C04DF
:100A800005FA04F61E4211D056070FD50A689206E1
:100A900003D40A6822F004020A6090F8441001F0BE
:100AA0001C018D40016C4D60016B1DE0022606FAB1
:100AB00004F71F424FF0000C4FF0010518D09707C4
:100AC00016D50A68920605D40A6822F00A020A605E
:100AD00080F8255090F8441001F01C018E40016C04
:100AE0004E6080F824C0C16A00291AD0F0BC0847C3
:100AF0000826A6401E4214D0120712D50A6822F01A
:100B00000E020A6090F84410026C01F01C0105FA14
:100B100001F15160C56380F8255080F824C0416B15
:100B2000E2E7F0BC7047000070B568B1334C016873
:100B30001423334AA14209D2324C0C44B4FBF3F3E0
:100B40009B00C0E910230BE0012070BD2B4C6442D8
:100B50000C44B4FBF3F39B004364284B083B036451
:100B6000022380F825300C6847F6F0739C43D0E9E7
:100B700002352B43D0E9045635432B4385692B437B
:100B8000C5692B43056A2B4323430B608168B1F58C
:100B9000804F29D0016C0F23914212D152F8A81F27
:100BA00090F8444004F01C04A3409943116090F86D
:100BB0004430416803F01C039940136819431160E5
:100BC00012E00E49A0310A6890F8444004F01C0479
:100BD000A3409A430A6090F84430426803F01C0333
:100BE0009A400B681A430A600021C163012280F811
:100BF000252080F82410084670BD0000080402403B
:100C000000000240F8FFFDBF70B5044690F82400D4
:100C1000002501280CD0012084F8240094F82560D8
:100C20000020012E06D084F824000225284670BD3D
:100C3000022070BD022684F82560E0632068066803
:100C400026F0010606602046FFF7B0FC206B002866
:100C50002068016802D041F00E0106E021F0040195
:100C600001602068016841F00A01016020680168A4
:100C700041F001010160D9E770B5044600F0D4F9F4
:100C80000546601C02D004480078044400F0CCF90A
:100C9000401BA042FAD370BD840000202DE9F05F14
:100CA000044632488946017801290CD00125804646
:100CB00005704CF2503B5846FFF7A0FD06004FF080
:100CC000000A03D04EE0022000F054B851464046DE
:100CD000C8F804A0264F3A6892050AD53968490534
:100CE00005D5396821F480613960032109E0057771
:100CF00008E03A68520504D5396821F4806139600A
:100D0000022101772068012807D04FF0FF31C9F890
:100D1000001040F2FA3BA5681DE06068FFF728FD6F
:100D20005846FFF76BFD0646786920F004007861AD
:100D300016E028466168FFF729FD4CF25030FFF7B6
:100D40005DFD0600786920EA0B00786102D0C9F8E1
:100D5000005005E06D1CD4E902010844A842E8D81F
:100D6000FFF7D8FC88F800A03046ADE790000020DF
:100D70000020024030BCBDE8C09F0000034841692C
:100D800041F0004141610020704700000020024016
:100D90002DE9FF5F254F05460024387891469B4694
:100DA000012809D0012038704CF25030FFF726FDA1
:100DB0000600A24604D035E0022004B000F03AB8A4
:100DC0005046C7F804A0DFF86880D8F8001049053D
:100DD00006D5D8F8001021F48061C8F80010022070
:100DE000387725B1012D09D0022D07D00DE04A46F4
:100DF0005B460198FFF7DEFC012406E049460198B6
:100E0000FFF7E6FC022D00D16C044CF25030FFF7E6
:100E1000F5FC064624B1D8F81410A143C8F8141004
:100E2000FFF778FC87F800A03046C6E79000002066
:100E30000020024030BCBDE8C09F000006490020F1
:100E40004A69002A07DA054A8A60054A8A604969C0
:100E5000002900DA01207047002002402301674585
:100E6000AB89EFCD2DE9F84FDFF880910022A9F191
:100E7000040B03274FF00F0C09F1040AABF1040E29
:100E8000ACE0012595402B4073D00C7904F00304AD
:100E9000012C01D0022C15D18668540007FA04F801
:100EA00026EA0806D1F80C8008FA04F848EA060891
:100EB000C0F808804468AC430D79C5F3001595402F
:100EC000254345600C79E443A40708D0C568540065
:100ED00007FA04F6B5438E68A6402E43C6600C7927
:100EE00004F00304022C11D1D40800EB8406356A07
:100EF0005407E40E0CFA04F825EA0805D1F810802E
:100F000008FA04F848EA0508C6F820800568540085
:100F100007FA04F6B5430E7906F00306A6402E4301
:100F200006604C6814F4403F57D0314C256E45F0B4
:100F300001052566246E22F0030504F001040094E7
:100F40002C4C05EB0408D8F808509407260F0CFA2F
:100F500006F4A543B0F1904F04D0274CA04203D132
:100F6000012412E0002410E0244CA04202D102240B
:100F70000BE032E0224CA04201D1032405E0214CD9
:100F8000A04201D1042400E00724B4402C43C8F857
:100F90000840D9F800404D464E689C43F60200D503
:100FA0001C432C60DAF8004055464E689C43B6025C
:100FB00000D51C432C60DBF800405D464E689C4326
:100FC000B60300D51C432C60DEF8004075464E6821
:100FD0009C43F60300D51C432C60521C0B6833FA6B
:100FE00002F47FF44EAF00F00FB800000804014097
:100FF00000100240000001400004004800080048C2
:10100000000C00480010004818BCBDE8E08F4269A1
:1010100021EA02030A4043EA0241816170470AB1B2
:1010200081617047816270470148806870470000A5
:101030008400002070B5040011D021684CF6CC402B
:101040000860216845F255500860D4E9000141600C
:101050002168A0688860FFF7E7FF05460CE00120E3
:1010600070BDFFF7E1FF401B312805D92068C0683B
:10107000400701D0032070BD2068C0684007F0D150
:1010800020680269E1688A4201D0016102E04AF603
:10109000AA210160002070BD00684AF6AA21016003
:1010A00000207047024881680278114481607047CF
:1010B0008400002010B50024032000F09FF80F20CA
:1010C00000F008F808B1012401E000F04FF82046D4
:1010D00010BD000030B505461F4887B0816D41F056
:1010E00010018165806D06A900F01000059068462A
:1010F00000F0D4FA0398B0B100F0F0FA40001749BC
:10110000174AB0FBF1F11748491E0260416040F2F6
:10111000E7320021C0E903218160816100F0FDFD1B
:10112000040003D015E000F0D9FAE8E70D4800F01C
:1011300027FE04000DD1362000F032F8102D07D222
:1011400000222946362000F039F80748056000E003
:10115000012407B0204630BD0010024040420F007D
:1011600000100040240E0020880000200B4882B0B0
:10117000016E41F001010166016E01F00101009173
:10118000816D41F080518165806D002200F08050BA
:1011900000900F21901E02B000F010B80010024025
:1011A000002809DB00F01F02012191404009800066
:1011B00000F1E020C0F8001170470000F0B40E4BC1
:1011C0001B68C3F30223C3F10704042C00D90424D1
:1011D0001D1D072D01D2002300E0DB1E012606FAAB
:1011E00004F56D1E0D409D409E40761E164045EA5A
:1011F0000601F0BC03F02AB80CED00E0064A00F04E
:10120000070110684FF6FF03184040EA0120034928
:1012100008431060704700000CED00E00000FA0584
:101220001649B0F5007F0868C0F3412009D00228B4
:1012300005D0086820F4C06040F480600860002099
:1012400070470128FBD0086820F4C06040F40070AB
:1012500008600B483222006850430A4AB0FBF2F0A3
:10126000401C00E0401E4A69520501D50028F9D112
:1012700048694005E3D50320704700000070004036
:10128000B000002040420F000248006800F4C06037
:1012900070470000007000402DE9F84F044600251B
:1012A0000088A64E2F46000515D5606C60B1B0F5DC
:1012B000000F04D0B0F5400F2BD001250AE0F068F4
:1012C00040F48030F06024E00021201D02F054F84A
:1012D00005001ED02F462068800365D5B06D4FF005
:1012E0000009C00009D4B06D40F08050B065B06D09
:1012F0004FF0010900F080500090DFF844A2DAF8C6
:10130000001041F48071CAF80010FFF78DFE80468E
:1013100010E0D6F88800616C20F440000843C6F85D
:101320008800D8E7FFF780FEA0EB0800022801D96B
:10133000032531E0DAF80000C005F3D565BBD6F827
:10134000900010F4407014D0A16D814211D0D6F8F5
:101350009000D6F8901020F4407041F48031C6F827
:101360009010D6F8901021F48031C6F89010C6F88D
:101370009000C0074ED0FFF757FE804641F2883AF2
:1013800005E0FFF751FEA0EB08015145D0D8D6F893
:1013900090008007F5D5EDB32F46B9F1000F03D0CB
:1013A000B06D20F08050B0652078C00707D0D6F827
:1013B0008800216A20F003000843C6F888002078DE
:1013C000800707D5D6F88800616A20F00C00084332
:1013D000C6F888002078400707D5D6F88800A16AAB
:1013E00020F030000843C6F888002078800607D532
:1013F000D6F88800E16A20F440600843C6F8880007
:101400002088800509D5D6F88800E16B20F44020BB
:10141000084300E044E0C6F888002088400507D56E
:10142000D6F88800216C20F440100843C6F88800E4
:101430002078400607D5D6F88800216B20F440506C
:101440000843C6F888002078000607D5D6F888003B
:10145000616B20F440400843C6F888002088C0052E
:1014600007D5D6F88800A16B20F440300843C6F8B1
:10147000880020684FF0006500034FF0806820D599
:10148000D6F88800A16C20F040600843C6F88800B8
:10149000A06CA8420DD1F06840F48010F06010E01C
:1014A000D6F89000A16D20F440700843C6F8900073
:1014B00073E7404505D10121201D01F05DFF00B11A
:1014C00007462068400317D5D6F88800E16C20F065
:1014D00040600843C6F88800E06CA84204D1F06878
:1014E00040F48010F06007E0404505D10121201D47
:1014F00001F042FF00B107462088400411D5D6F81C
:101500008800216D20F040500843C6F88800206D07
:10151000B0F1805F05D10221201D01F02DFF00B147
:1015200007462088000406D556F8880F616D20F024
:10153000804008433060384600F004B80010024094
:101540000070004018BCBDE8E08F00002DE9F047B6
:101550000D46040071D0DFF83081D8F8000000F0AB
:101560000700A8420CD2D8F8001021F00701294347
:10157000C8F80010D8F8000000F00700A8425CD1BD
:101580002078424E80070AD5A068B16801F0F001CA
:10159000884204D9B16821F0F0010143B16020789C
:1015A000C0072BD06068032811D0022812D0316800
:1015B00098B14905002940DAB16821F003010143DF
:1015C000B160FFF731FD074641F288390FE031681D
:1015D0008901EFE731688903ECE78907EAE7FFF75C
:1015E00023FDC11B494502D90320BDE8F087B0683F
:1015F000616800F00C00B0EB810FF0D1207880071B
:101600000AD5A068B16801F0F001884204D2B1683F
:1016100021F0F0010143B160D8F80010404601F01C
:101620000701A9420BD9016821F007012943016094
:10163000006800F00700A84201D00120D5E720781B
:10164000400705D5B068E16820F4E0600843B06069
:101650002078000706D5B068216920F4605040EA80
:10166000C100B06000F05EF8B168094AC1F303112F
:10167000515C01F01F01C840064908600648006837
:10168000BDE8F047FFF726BD0020024000100240F1
:10169000AC660008B0000020880000200F22026025
:1016A0000C4A936803F003034360936803F0F0036C
:1016B0008360936803F4E063C36092684FF4E0636F
:1016C00003EAD20202610448006800F007000860E3
:1016D0007047000000100240002002400548064903
:1016E00000688968054AC1F30221515C01F01F01BD
:1016F000C8407047B000002000100240EC660008AF
:101700000548064900688968054AC1F3C221515C51
:1017100001F01F01C8407047B000002000100240D7
:10172000EC66000870B5254B002210469968DC680D
:1017300011F00C0104F00306214C4FEA640508D0B7
:101740000C2904D0042931D0082931D010E0012E11
:1017500010D11A68120704D4D3F89420C2F30322DC
:1017600002E01A68C2F30312164E56F82220D9B1CD
:101770000C2918D1D86800F0030002281AD00328D9
:101780001AD01046D968DA68C1F30211C2F30622F2
:101790004243491CB2FBF1F0D968C1F34161491CD5
:1017A0004900B0FBF1F070BD104670BD204670BD21
:1017B000284670BD2046E5E72846E3E700100240D2
:1017C0000024F400BC6600082DE9F84304006FD043
:1017D000F64EB06800F00C05F06800F003072078C2
:1017E000C00664D575B10C2D01D1012F0AD0A069B6
:1017F0000028306879D040F001003060FFF714FC19
:1018000080465CE03068800702D5A0690028DED001
:10181000216A3068000703D5306800F0F00004E06A
:10182000D6F89400F02202EA1010814216D9084638
:1018300001F036FE00283BD1306840F008003060EF
:101840003068216A20F0F000084330607068E16978
:1018500020F47F4040EA0120706016E0306840F0DC
:10186000080030603068216A20F0F00008433060E2
:101870007068E16920F47F4040EA0120706025B97A
:10188000206A01F00DFE0028D5D1FFF74BFFB168AB
:10189000C74AC1F30311515C01F01F01C840C5499B
:1018A0000860C5480068FFF715FC00287ED12CE0D1
:1018B000C6E0FFF7B9FBA0EB0800022877D8306834
:1018C0008007F6D5306840F0080030603068216A43
:1018D00020F0F000084330607068E16920F47F4038
:1018E00040EA0120706010E0FFE720F00100306066
:1018F000FFF79AFB804605E0FFF796FBA0EB080098
:101900000228DBD830688007F6D42078C00740D0A2
:10191000082D18D00C2D01D1032F14D06068B0F51C
:10192000803F17D0B0F5A02F306817D020F480305A
:101930003060306820F4802030606068E0B1FFF7EC
:1019400073FB804614E03068800322D5606800286D
:1019500076D01EE0306840F48030EDE740F480201F
:101960003060F7E7FFF760FBA0EB08006428A5D81C
:1019700030688003F6D50CE0FFF756FB804605E0A3
:10198000FFF752FBA0EB0800642897D8306880036B
:10199000F6D42078800739D5042D11D00C2D01D133
:1019A000022F0DD0E0680028306801E0A0E1FBE0E4
:1019B0001DD040F480703060FFF736FB07460BE027
:1019C000306840050BD5E0680028C1D007E0FFF77C
:1019D0002BFBC01B022894D830684005F7D57068EF
:1019E000217C20F0F85040EA016070600EE020F4A5
:1019F00080703060FFF718FB074604E0FFF714FB28
:101A0000C01B0228B3D830684005F7D420780007FF
:101A100028D560690028D6F8940012D040F0010063
:101A2000C6F89400FFF700FB074604E0FFF7FCFA56
:101A3000C01B02289BD8D6F894008007F6D511E089
:101A400027E120F00100C6F89400FFF7EDFA074601
:101A500004E0FFF7E9FAC01B022888D8D6F8940002
:101A60008007F6D42078400765D5B06D4FF00008A8
:101A7000C00009D4B06D40F08050B065B06D4FF03B
:101A8000010800F0805000904C480168C90511D44D
:101A90000168814641F480710160FFF7C5FA07468D
:101AA00004E0FFF7C1FAC01B02287DD8D9F8000076
:101AB000C005F6D5A068012815D00528D6F89000F5
:101AC00016D020F00100C6F89000D6F8900020F063
:101AD0000400C6F89000A06841F28839B8B1FFF759
:101AE000A3FA07460EE0D6F8900040F00100F0E7B8
:101AF00040F00400C6F89000F5E7FFF795FAC11B27
:101B0000494551D8D6F890008007F6D50CE0FFF78C
:101B10008BFA074604E0FFF787FAC11B494543D813
:101B2000D6F890008007F6D4B8F1000F03D0B06D5E
:101B300020F08050B0652078800627D5606A0028A4
:101B4000D6F8980011D040F00100C6F89800FFF7D1
:101B50006BFA074604E0FFF767FAC01B022823D898
:101B6000D6F898008007F6D510E020F00100C6F8FE
:101B70009800FFF759FA074604E0FFF755FAC01B33
:101B8000022811D8D6F898008007F6D4A06AE8B3E6
:101B9000022815D00C2D7CD0306820F08070306089
:101BA000FFF742FA0446A5E0A1E000000010024061
:101BB000AC660008B00000208800002000700040E3
:101BC000F068E26A00F00301914228D1216B00F035
:101BD000700209011039914221D1626B00F4FE417B
:101BE000B1EB022F1BD194F8382000F07841B1EB13
:101BF000C26F14D1A18F00F4C00249084905A1F5B4
:101C0000001191420BD194F8401000E069E04908BE
:101C1000490600F0C060A1F1007181424AD00C2D4C
:101C200071D0306840016ED4306820F08070306030
:101C3000FFF7FAF9054604E0FFF7F6F9401B022822
:101C400055D830688001F7D4F4E90B016FF00F022A
:101C500002EB01110843218A5204490802EB415169
:101C6000A26841EA02210843217D4FF07E424908E3
:101C700002EB41610843217B40EAC160F168234ADD
:101C800011400843F060306840F080703060F068C8
:101C900000E038E040F08070F060FFF7C5F90446DE
:101CA00004E0FFF7C1F9001B022820D8306880014A
:101CB000F7D526E03068800123D4306840F080708A
:101CC0003060F06840F08070F060FFF7ADF90446D6
:101CD00004E0FFF7A9F9001B022808D8306880014A
:101CE000F7D50EE0FFF7A0F9001B022802D9032068
:101CF000BDE8F88330688001F4D4F06804490840F6
:101D0000F0600020F4E70120F2E700008C809D01E4
:101D1000FCFFEEFE70477047704710B5040003D01B
:101D200094F83D0010B107E0012010BD002084F8B8
:101D30003C00204600F022F8022084F83D00211DDE
:101D4000206801F037FE012084F8480084F83E0046
:101D500084F83F0084F8400084F8410084F8420091
:101D600084F8430084F8440084F8450084F8460071
:101D700084F8470084F83D00002010BD7047000043
:101D800090F83D10012901D001207047022180F810
:101D90003D100168CA6842F00102CA6000680B4940
:101DA000884205D0B0F1804F02D00949884207D15E
:101DB0008168084A1140062906D0B1F5803F03D05A
:101DC000016841F00101016000207047002C0140D2
:101DD0000040014007000100704770B504460068EC
:101DE00001694FF00005C943890715D4C168C9438B
:101DF000890711D4E91E01610120207720688069DC
:101E00008007204602D0FFF7E7FF04E000F0A7F8C4
:101E1000204600F0A5F8257720680169C9434907E5
:101E200017D4C168C943490713D46FF00401016195
:101E3000022020772068806910F4407F204602D07D
:101E4000FFF7CAFF04E000F08AF8204600F088F8A7
:101E5000257720680169C943090716D4C168C943B9
:101E6000090712D46FF0080101610420207720686F
:101E7000C0698007204602D0FFF7AEFF04E000F003
:101E80006EF8204600F06CF8257720680169C94398
:101E9000C90617D4C168C943C90613D46FF010012D
:101EA0000161082020772068C06910F4407F204637
:101EB00002D0FFF791FF04E000F051F8204600F057
:101EC0004FF8257720680169C943C90708D1C1685F
:101ED000C943C90704D1891E0161204600F042F8B8
:101EE00020680169C943090609D4C168C9430906C4
:101EF00005D46FF0800101612046FFF70CFF2068D8
:101F00000169C943C90509D4C168C943090605D493
:101F10006FF4807101612046FFF7FCFE20680169C3
:101F2000C943490609D4C168C943490605D46FF0BD
:101F300040010161204600F01FF820680169C94393
:101F400089060BD4C168C943890607D46FF0200104
:101F500001612046BDE87040FFF7DEBE70BD7047EE
:101F60007047000000680349884201D1FFF79AB822
:101F7000704700000010004070477047704770B510
:101F80000446806FE66F216889684FF010050906E6
:101F900018D5212816D12068083050E8001F21F0FC
:101FA000800140E80012002AF5D1E06E38B1FEF75A
:101FB0000FFD20B1E06EFEF757FD202821D020460E
:101FC00001F009FF20688068400618D5222E16D13E
:101FD0002068083050E8001F21F0400140E800125E
:101FE000002AF5D1206F38B1FEF7F2FC20B1206F46
:101FF000FEF73AFD202804D0204601F0C7FE00205D
:1020000070BDC4F88050032070BD70472DE9F041C9
:1020100002680446D0691168966840F60F031842BA
:102020004FF0000505D183067ED58B067CD5616E09
:102030001BE1994F06F001030F401F4374D0C707FF
:1020400009D0CF0507D501271762D4F8802042F0C8
:102050000102C4F8802082070AD5F20708D0276859
:1020600002223A62D4F8802042F00402C4F88020B0
:1020700042070AD5F20708D0266804223262D4F853
:10208000802042F00202C4F8802002070CD501F043
:1020900020021A4308D0236808221A62D4F880204C
:1020A00042F00802C4F8802002050BD54A0109D588
:1020B00023684FF400621A62D4F8802042F02002B4
:1020C000C4F88020D4F88020002A35D0800605D5B9
:1020D000880603D5616E09B120468847D4F8800090
:1020E00021688968490602D410F0280F26D02046BE
:1020F00001F04CFE2068806840061AD52068083040
:1021000050E8001F21F0400140E80012002AF5D1FC
:10211000206F70B161498163206FFEF77EFC00285B
:102120000AD0206F816B01E00EE02046BDE8F0414F
:1021300008472046FFF769FFBDE8F0812046FFF71A
:1021400064FFC4F88050F7E7276E2023012F7BD16E
:10215000C70679D5CF0677D5102010622068806831
:10216000400641D5216F086840680004000CE3D0A8
:10217000B4F858208242DFD9A4F85A0008680068F1
:1021800080062AD4206850E8001F21F4807140E8BE
:102190000012002AF6D12068083050E8001F21F014
:1021A000010140E80012002AF5D12068083050E80B
:1021B000001F21F0400140E80012002AF5D1E3673A
:1021C0002566206850E8001F21F0100140E8001249
:1021D000002AF6D1206FFEF7FBFBB4F85800B4F8E4
:1021E0005A10401A81B22AE0B4F85800B4F85A10D4
:1021F000401A81B2B4F85A0000289DD000299BD023
:10220000206850E8002F22F4907240E80026002E4B
:10221000F6D12068083050E8002F22F0010240E893
:102220000026002EF5D1E36725666566206850E834
:10223000002F22F0100240E80023002BF6D12046A8
:10224000FFF79BFE78E7FFE7C70209D5760207D5BF
:102250004FF4801010622046BDE8F041FFF78EBEBB
:10226000020606D50A0604D5A16E00297FF45DAFEB
:1022700062E74006E6D54806E4D52046016851E805
:10228000002F22F0400241E80024002CF6D18367A1
:10229000856600F0B5F94FE720010004453C0008D1
:1022A00010B5040002D0A06F10B107E0012010BDEE
:1022B000002084F87400204600F026F82420A0674F
:1022C0002068016821F001010160204601F090FDC5
:1022D0000128ECD0606A10B1204601F021FC206892
:1022E000416821F4904141602068816821F02A0111
:1022F00081602068016841F0010101602046BDE86D
:10230000104001F071BC00002DE9F0439DB004467F
:10231000142117A8FEF715F85C216846FEF711F89E
:1023200046492068464E022700254FF003084FF02B
:10233000070988425BD10120009008956846FEF7A6
:10234000ABFF08B1FEF7E4F9306E40F48040306630
:10235000306E00F480401C90F06C40F00100F0649E
:10236000F06C19AA00F001001C904FF4C060CDE998
:10237000170782E8200317A94FF09040FEF772FD7F
:10238000314E30484FF080083060C6E90175C6E92B
:1023900003587561B561F56130463562FEF7C4FBDF
:1023A00008B1FEF7B5F92667B462274E25484836CE
:1023B0001438E6E802071020A6E82101224846F872
:1023C00014594830B561F5613562FEF7ADFB08B1CF
:1023D000FEF79EF9E666002205212520B462FEF78D
:1023E000EDFE2520FEF7DCFE1DB0BDE8F0831749A9
:1023F0008842F9D104200A9500906846FEF74CFF08
:1024000008B1FEF785F9B06D40F48020B065B06D7D
:1024100000F480201C90F06C40F00400F064F06C3C
:1024200019AA00F004001C903020CDE9170782E8BB
:10243000200317A90648FEF715FDD5E7003801402F
:102440000010024058000240940D00200048004057
:102450000008004830B4C36F202B20D1E1B1DAB1BD
:1024600090F87430012B1AD0012380F874300023C7
:1024700003660C4C0368A3420BD05B681B0208D5B3
:10248000036853E8004F44F0806443E80045002DA2
:10249000F6D130BC01F0AABD012030BC704702204B
:1024A000FBE7000000800040704770472DE9F843CB
:1024B0000446806F1F4615460E4620284ED1CEB1E9
:1024C000C5B194F87400012848D0012084F8740044
:1024D0004FF00008C4F880802120A067FEF7A4FD1B
:1024E000A4F850508146A4F85250A068B0F5805F1F
:1024F00003D004E00120BDE8F883206920B135460F
:10250000002684F8748010E00025FAE78021204638
:1025100001F0BEFDB8B9C5B115F8010B21680885F9
:10252000B4F85200401EA4F85200B4F852004B46D2
:102530004FF0000200970028E8D14FF040012046FC
:1025400001F0A6FD30B10320D5E736F8020BC0F349
:102550000800E3E72020A0670020CCE70220CAE7BC
:1025600070B50446806F202841D169B362B394F8F6
:10257000740001283BD0012084F87400E164A4F8C1
:102580005020A4F852200025C4F880502120A067D4
:10259000E06ED8B11749C162E16E1748134608636F
:1025A000E16E16484863E06E85632668E16C06F1CB
:1025B0002802E06EFEF728FB40B11020C4F880002E
:1025C00004F8745F20206060012070BD2168402005
:1025D000086284F874502068083050E8001F41F009
:1025E000800140E80012002AF5D1002070BD0220D1
:1025F00070BD0000413D0008833D0008593C0008C3
:1026000070477047FEE7000070B50E4C00230126AE
:10261000E260E38003780725402B05D143783BB186
:10262000012B08D0022B09D01570E680E08870BD20
:10263000FDF7D4FFFAE701F0F3F9F7E701F03EFA0E
:10264000F4E700005400002004484178012903D039
:1026500003490161012141707047000054000020CE
:1026600000000308F0B585B0174D002404946C7089
:10267000164928690844B0F5803F02D3081705B011
:10268000F0BDFEF7DBFB00942869FEF7F5F8029039
:1026900001200190039004A96846FEF7FFFA0C4E52
:1026A000002406EBC400D0E90023286900EBC40134
:1026B0000020FEF76DFB641C0746FF2CF1DDFEF7E2
:1026C0005DFB3846DBE70000540000200000FDF70A
:1026D000580200202DE9F04F064687B000202C4F0D
:1026E000CDE9040082467878DFF8A8900D464FF4D3
:1026F000006B012806D147E0274938690844B0F546
:10270000803F04D34FF0FF3007B000F047B878693E
:10271000D8464119414503D9C0F500618CB200E0AB
:102720002C46484422463146FDF7F2FD7869291BC4
:10273000204426448DB27861404525D1FEF77EFBCA
:10274000CDF800A0D0463869FEF796F80290012037
:102750000190039005A96846FEF7A0FA002409EB52
:10276000C400D0E90023386900EBC4010020FEF763
:102770000FFB641C0490FF2CF1DDFEF7FFFA3869B3
:1027800000F50060C7E90408002DB5D10498BBE747
:1027900054000020580200200000FDF730BCBDE8C6
:1027A000C08F000010B50DA001F040FD124908686F
:1027B000124A1040B0F1005F04D0BDE8104010A0F4
:1027C00001F034BD012080F3108848681A4AD061B6
:1027D000096881F30888BDE8104000473E20494160
:1027E00050204A756D70544F4170703120202E2E4C
:1027F0002E2E2E2E0D0A0000000002080000FE2FD3
:10280000746F70206F6620737461636B20706F69E2
:102810006E74657220697320756E76616C696421CF
:1028200020656E746572204150502075706461742B
:1028300065210D0A00000000540000207CB50C4604
:102840000546082210316846FDF749FF208AC0F38B
:10285000C502382A02D2C2F1380201E0C2F1780280
:102860000949204600F097FB08226946204600F0FF
:1028700092FB102221462846FDF731FF5822002105
:10288000204600F0C9FB7CBD000000200021416112
:10289000016105490160054941600349C9438160FF
:1028A0000249C943C16070470123456789ABCDEF39
:1028B0002DE9F04F50F804BB002590E8580091B086
:1028C000EA464FF040092A46001F8F18121D97F85C
:1028D0000280B7F800C0FF7868F31F4C4CEA076C21
:1028E0004AF825C06D1C4A45EFD303EA040126EAE5
:1028F00003021143FE4A009D0A4405EB0B011144FB
:1029000003EB716202EA030124EA02073943F94F3B
:102910003944019F3E44314402EB315101EA020641
:1029200023EA01073E43F44F3E44029F3C443444B3
:1029300001EBF43404EA010622EA04073E43EF4FB8
:102940003E44039F3B44334404EBB32303EA0406B1
:1029500021EA03073E43EA4F3E44049F3A4432448F
:1029600003EB726202EA030624EA02073E43E54FE4
:102970003E44059F3944314402EB315101EA0206DD
:1029800023EA01073E43E04F3E44069F3C44344463
:1029900001EBF43404EA010622EA04073E43DB4F6C
:1029A0003E44079F3B44334404EBB32303EA04064D
:1029B00021EA03073E43D64F3E44089F3A4432443F
:1029C00003EB726202EA030624EA02073E43D14F98
:1029D0003E44099F3944314402EB315101EA020679
:1029E00023EA01073E430A9FA6F524463C444F3E96
:1029F000344401EBF43404EA010622EA04073E43BE
:102A0000C54F3E440B9F3B44334404EBB32303EADE
:102A1000040621EA03073E43C04F3E440C9F3A445C
:102A2000324403EB726202EA030624EA02073E43E1
:102A3000BB4F3E440D9F3944314402EB315101EA12
:102A4000020623EA01073E43B64F3E440E9F3C4434
:102A5000344401EBF43404EA010622EA04073E435D
:102A6000B14F3E440F9F3B44334404EBB32303EA8E
:102A7000010624EA01073E43AC4F3E44019F3A441D
:102A8000324403EBF26202EA040623EA04073E43FF
:102A9000A74F3E44069F3944314402EBF15101EA0D
:102AA000030622EA03073E43A24F2B443E440B9FFA
:102AB0003C44344401EBB44404EA020621EA020730
:102AC0003E439D4F3E44334404EB333303EA010657
:102AD00024EA01073E43994F3E44059F3A4432445D
:102AE00003EBF26202EA040623EA04073E43944F32
:102AF0003E440A9F3944314402EBF15101EA030696
:102B000022EA03073E438F4F3E440F9F3C44344428
:102B100001EBB44404EA020621EA02073E438A4F6D
:102B20003E44049F3B44334404EB333303EA010641
:102B300024EA01073E43854F3E44099F3A4432440C
:102B400003EBF26202EA040623EA04073E43804FE5
:102B50003E440E9F3944314402EBF15101EA030631
:102B600022EA03073E437B4F3E44039F3C443444E8
:102B700001EBB44404EA020621EA02073E43764F21
:102B80003E44089F3B44334404EB333303EA0106DD
:102B900024EA01073E43714F3E440D9F3A443244BC
:102BA00003EBF26202EA040623EA04073E436C4F99
:102BB0003E44029F3944314402EBF15101EA0306DD
:102BC00022EA03073E43674F3E44079F3C44344498
:102BD00001EBB44404EA020621EA02073E43624FD5
:102BE0003E440C9F3B443344059E04EB3333164470
:102BF00083EA04025D4F4A403A443244089E03EBA4
:102C000032720E4482EA0301594F61403944314423
:102C100002EB71560B99574F0C4486EA020159405A
:102C20003944214406EB31440E99534F0B4484EA56
:102C30000601514039441944019B04EB71211344AE
:102C400081EA04024D4F72403A441A44049B01EB5E
:102C500032721E4482EA0103494F63403B443344CD
:102C600002EB7356079B474F1C4486EA02034B4016
:102C70003B4423440A9C06EB33430C4483EA06019D
:102C8000414F5140394421440D9C03EB71211444C0
:102C900081EA030272403D4F2E443A44224401EB44
:102CA000327282EA01043A4F5C403C443444039E51
:102CB00002EB74541E4484EA0203364F4B403B44FB
:102CC0003344069E04EB33430E4483EA0401324F3F
:102CD000514039443144099E03EB7121164481EA85
:102CE00003022E4F62403A44324401EB327257E005
:102CF00078A46AD756B7C7E8DB702024EECEBDC1F2
:102D0000AF0F7CF52AC68747134630A8019546FDCC
:102D1000D8988069AFF7448BBED75C892211906B3D
:102D2000937198FD8E4379A62108B44962251EF659
:102D300040B340C0515A5E26AAC7B6E95D102FD6EF
:102D40005314440281E6A1D8C8FBD3E7E6CDE121C4
:102D5000D60737C3870DD5F4ED145A4505E9E3A925
:102D6000F8A3EFFCD9026F678A4C2A8D4239FAFF2B
:102D700081F6718722619D6D0C38E5FD44EABEA4A1
:102D8000A9CFDE4B604BBBF670BCBFBEC67E9B2896
:102D9000FA27A1EA8530EFD4051D880439D0D4D9AB
:102DA0000C9E684F264482EA01045C403C44344453
:102DB0000F9E02EB74541E4484EA0203624F4B40A0
:102DC0003B443344029E04EB33430E4483EA040144
:102DD0005E4F51403944314403EB7121154461EA9F
:102DE00004025B4E5A4032442A44079D01EBB26212
:102DF000254462EA0304574E4C4034442C440E9D53
:102E000002EBB4541D4464EA0103534E534033446F
:102E10002B44059D04EB73430D4463EA02014F4EBE
:102E20006140314429440C9D03EBF121154461EAD2
:102E300004024B4E5A4032442A44039D01EBB262D5
:102E4000254462EA0304474E4C4034442C4402EBD0
:102E5000B4550A9C1C4465EA01035340424E334476
:102E6000234405EB7344019B404E0B4464EA02018A
:102E700069403144194404EBF12308993C4E0A445B
:102E800063EA05016140314411440F9A03EBB161DB
:102E9000154461EA0402374E5A4032442A44069DE2
:102EA00001EBB252254462EA0304334E4C403444F1
:102EB0002C440D9D02EB74441D4464EA01032F4E23
:102EC000534033442B44049D04EBF3230D4463EA45
:102ED00002012B4E6140314429440B9D03EBB1614B
:102EE000154461EA0402274E5A4032442A44029DA6
:102EF00001EBB252254462EA0304234E4C403444B1
:102F00002C44099D02EB74441D4464EA01031F4EE6
:102F1000534033442B44056804EBF32329440160F8
:102F2000416819444160816821448160C16811444D
:102F3000C16040220021504600F06EF811B000F050
:102F400027B80000E599DBE6F87CA21F6556ACC403
:102F5000442229F497FF2A43A72394AB39A093FC7A
:102F6000C3595B6592CC0C8F7DF4EFFFD15D8485F6
:102F70004F7EA86FE0E62CFE144301A3A111084E7A
:102F8000827E53F735F23ABDBBD2D72A91D386EB76
:102F900030BCBDE8C08F2DE9F0410F460169054600
:102FA0001646C1F3C50001EBC6012961B1EBC60F9E
:102FB000696901D2491C696101EB5671C0F1400495
:102FC0006961A64216D3284422463946183000F0DB
:102FD0001AF805F118012846FFF76AFC04E03919D0
:102FE0002846FFF765FC403404F13F00B042F6D3B9
:102FF000002000E00024321B39192844BDE8F041CC
:103000001830AFF3008010B5002302E0CC5CC4544C
:103010005B1C9342FAD310BD0023C9B201E0C15436
:103020005B1C9342FBD370470F4810B50D490160FC
:1030300001210171417148F2050282600822C260DB
:103040004FF6FF720261202242618022826101629A
:10305000FDF770FC002803D0BDE81040FDF758BB19
:1030600010BD000000300240880A00200D4808B55D
:10307000816C41F001018164806C002200F001004C
:10308000009005210E20FEF799F80E20FEF788F833
:10309000002205210F20FEF791F8BDE808400F201F
:1030A000FEF77EB80010024010B50FA001F0BEF888
:1030B000134A0021134801F097FD134C104A0021D8
:1030C00020602432114801F08FFD0D4A60604832C3
:1030D00000210F4801F088FDA06009486C3001F024
:1030E0003EFDE06010BD0000204D585F4652454552
:1030F00052544F535F496E697420200D0A0000003E
:10310000306600087136000874000020BD360008E3
:10311000DD36000870B586B014216846FDF711F958
:103120003448C16C41F00401C164C16C01F0040178
:103130000591C16C41F08001C164C16C01F0800156
:103140000591C16C41F00101C164C16C01F0010144
:103150000591C16C41F00201C164C16C01F0020132
:103160000591C16C41F00801C164C06C224E00F0B1
:103170000800059000220F213046FDF750FF4FF662
:10318000C0700325CDE9000500246946029430464D
:10319000FDF768FE0F2000900120CDE9010469468B
:1031A00030460394FDF75EFE49F6FF10CDE90005B9
:1031B000694602944FF09040FDF754FE4FF6FF70C1
:1031C000CDE90005694602940C48FDF74BFE04204A
:1031D000CDE90005694602940948FDF743FE082041
:1031E000CDE90005694602940648FDF73BFE06B0AE
:1031F00070BD0000001002400008004800040048B4
:10320000000C0048001C00480A4810B5084901603D
:103210000321416040F2E731C1608160FDF70AFFA0
:10322000002803D0BDE81040FDF772BA10BD0000C1
:1032300000300040AC0A002070B5224C20482060CD
:1032400021480068C1784FF41650082907D2DFE8FA
:1032500001F0060406272A2D30334FF4965000253E
:10326000C4E901050C20E560C4E90450A561E561ED
:10327000256214486562FFF713F808B1FDF748FAB4
:10328000124800F110010573416000F5A8718160DA
:10329000058045802068016841F01001016070BD23
:1032A0004FF49640DBE74FF41640D8E74FF4614007
:1032B000D5E74FF4E130D2E74FF46130CFE70000BB
:1032C000003801408C0C002040000020BC0A002087
:1032D0000D4810B50B4901604FF4E1314160002108
:1032E00081600C22C160C0E904128161C161016288
:1032F0004162FEF7D5FF002803D0BDE81040FDF77E
:1033000007BA10BD00480040100D0020FEE7000085
:1033100070B5144A144C506820601188218192685D
:1033200062608022A28100226281A273022911D9E7
:103330000E4A126893780278934201D0FF2A09D18D
:103340004218891E32F8025C01F0B4FBA84201D198
:1033500001F0DCFB2089002803D0BDE8704002F0BA
:10336000DDB870BDBC0A00203801002040000020FC
:1033700002F0D4B8FEE700002DE9F041434E0546C7
:103380008846F0680024810728680ED0F16801F0B3
:103390000301814207D130B1F0686968C0F30210BF
:1033A000401C88421FD001246DE0012809D002286A
:1033B0000AD00328F7D13168890309D43168490359
:1033C00004E03168890701E0316849050029EADA3B
:1033D000F1686A686FF00F0321F0730103EB0212CA
:1033E00011430143F160306820F080603060FDF7E8
:1033F0001BFE074604E0FDF717FEC01B022838D865
:1034000030680001F7D474BBB8F1000F18D0B8F1E0
:10341000010F1DD0287D4FF07E41400801EB406038
:10342000A96840EA01203169194A11400843306116
:10343000306840F080603060FDF7F6FD07461AE026
:10344000A868297B000240EAC1603169114AECE7B3
:10345000288A1149400801EB4050A96840EA012040
:1034600031690E4AE1E70EE0FDF7DEFDC01B0228E0
:1034700001D9032407E030680001F5D51CB9306993
:10348000A969084330612046BDE8F0810010024080
:10349000FF80FFF9FF80FF070000E0FFFF809FFF34
:1034A000F8B51C4E05460024B06DC00002D5FDF7EE
:1034B000EBFE0DE0B06D40F08050B065B06D00F0F7
:1034C00080500090FDF7E0FEB16D21F08051B165B4
:1034D000B0F5007F04D0802D07D94FF003040AE037
:1034E000802D08D9A02D01D804E001D1022402E0EA
:1034F000702D00D101240848016821F00701214303
:103500000160006800F00700A04201D00120F8BD72
:103510000020F8BD0010024000200240022901D224
:1035200000207047002101700249096889784170C4
:103530000220704740000020022901D2002070477D
:103540000021017002490968C97841700220704762
:1035500040000020042901D2002070470A490A686F
:10356000D2F8F020120E02700A68D2F8F020120C85
:1035700042700A68B2F8F020120A8270096891F865
:10358000F010C1700420704740000020022901D2D1
:103590000020704705490A68B2F8EE20120A02704E
:1035A000096891F8EE104170022070474000002039
:1035B00010B5102901D2002010BD0C4B002153F88A
:1035C0002120120E00F8212053F82120140C00EBCA
:1035D0008102547033F82140240A947013F821407A
:1035E000491CD4700429EADB102010BD44000020DF
:1035F000022901D20020704705490A68B2F8EC2080
:10360000120A0270096891F8EC10417002207047AC
:103610004000002010B5FDF723F9002010BD000088
:10362000F0B585B000240494FDF708FC202002903A
:103630000120CDE9004003900B4D04A96846FDF739
:103640002DFB0A4E05EBC40106EBC400D0E90023B4
:103650000020FDF79DFB641C0746212CF2D3FDF7EB
:103660008DFB05B03846F0BD000001085001002078
:1036700000240A4F0A4D4FF4FA76304602F0A8F8BB
:1036800001213846FDF7C3FC214606A000F0CEFD1F
:103690000121E86802F002FA641CEEE70008004825
:1036A0007400002074686520626F6F7420636F750A
:1036B0006E743A205B25645D200D0A00FFF758FE0A
:1036C000054CFFF725FE322001F03CFA0221E068AC
:1036D00002F0E4F9F5E700007400002008B5084C9A
:1036E0004FF0FF35012300951A460321E06802F0F0
:1036F0001BFA00F04DFF642001F024FAF2E700000D
:10370000740000202DE9F04F85B0DFF874A100248B
:103710000494DAF80000DFF86C81B0F8FC0000F6E1
:103720004520B0F5C04073D000F61130B0F5C04070
:103730000AD000F6EF60B0F5005F02D152A000F0B1
:1037400075FD05B000F0DEB856A000F06FFDDAF8A8
:103750000000D0F8F810B1F5803F72D856465848AE
:10376000FCF756FE00286CD03068B246DFF8549162
:10377000D0F8F86000254FF0010B4FF4006296423C
:103780002CD34F4829184F48FCF7C2FDFDF756FBD4
:10379000002047460090E819FDF76EF8CDE901B02A
:1037A00004A96846CDF80CB0FDF778FA0024B846B5
:1037B00009EBC40005EBC401D0E90023414400201B
:1037C000FDF7E6FA641C0746FF2CF1DDFDF7D6FA9B
:1037D00005F50065B6F50066CFD12BE038483246D6
:1037E00029183848FCF794FDFDF728FB00200090CD
:1037F00005EB0800FDF740F8CDE901B004A96846E3
:10380000CDF80CB0FDF74AFA00240746F61D0CE08F
:103810001FE009EBC40005EBC401D0E900234144DB
:103820000020FDF7B5FA0746641CB4EBD60FF0D3C1
:10383000FDF7A4FA2FB9DAF80000D0F8F810C0F8B4
:10384000F410DAF8000045F2BB51A0F8FC10FFF7C5
:10385000E7FE1DA000F0EAFCDAF80000D0F8F41052
:10386000B1F5803F3FF66DAF4046FCF7D1FD002833
:103870003FF467AF1BA000F0D9FCFEF793FF60E7B1
:1038800040000020000002083E20494150204E6FB9
:10389000726D616C2073746172742E2E2E2E2E2E1A
:1038A0000D0A00003E204941502055706461746546
:1038B0002073746172742E2E2E2E2E2E0D0A00008F
:1038C00000000308580200203E2049415020537454
:1038D00061727475702061707031202E2E2E2E2E24
:1038E0002E0D0A003E2049415020537461727475B8
:1038F00070206170703120323232202E2E2E2E2E0A
:103900002E0D0A0030BCBDE8C08F10B54FF0E0208E
:10391000006902F0DDFC012803D0BDE8104002F090
:1039200001BA10BD10B596B044216846FCF709FDF8
:10393000142111A8FCF705FD4FF40070FDF770FC91
:1039400008B172B6FEE7092000904FF480300121E3
:1039500001900591022003240A90CDE90B41142126
:103960000D910721CDE90E1010906846FDF72CFF50
:1039700008B172B6FEE70F20CDE9110400201390C4
:1039800014901590042111A8FDF7E0FD002801D046
:1039900072B6FEE716B010BD0248016841F470012E
:1039A0000160704788ED00E00148FEF716BA00009C
:1039B000240E0020F0B50268164C4FF08047A0425C
:1039C00001D0B84203D122F070034A681A43124D65
:1039D000124EA04205D0B84203D0A84201D0B04256
:1039E00003D122F44073CA681A434B6922F0800263
:1039F0001A4302608A68C2620A688262A04203D0E7
:103A0000A84201D0B04201D109690163012141619D
:103A1000F0BD0000002C0140004001400044014086
:103A20002DE9F0410D4681784FF6FF7202EA01213F
:103A3000C278214C11448FB2E288E168412300260C
:103A40008B54521C92B22B1F8E54521C92B2E280A5
:103A5000B3F5807F01DD022004E0B4F804C06745BF
:103A600004D004208854521CE2800AE099B2001D60
:103A7000FEF730FE40B1E088E26808211154401C96
:103A8000E080FEF7EFFD0BE0E088E1680E54401C9B
:103A9000E080A0682844001FA060A088401CA0808F
:103AA000A188E088E2680B0A1354401C80B21154CC
:103AB000401CE080BDE8F0815400002070B5164C39
:103AC00041220025E088E1680A54401C80B20D5470
:103AD000401CE080FEF7C6FD08B1082104E0A169A2
:103AE000A068884206D00321E088E2681154401C97
:103AF000E08070BDE088E2681554401CE080074813
:103B0000006840F8F81F4AF6AA218180FFF788FD77
:103B10000120207070BD00005400002040000020F3
:103B200090F82410C90706D001684A68836A22F415
:103B300000321A434A6090F82410890706D50168BC
:103B40004A68C36A22F480321A434A6090F824100B
:103B5000490706D501684A68036B22F480221A439C
:103B60004A6090F82410090706D501684A68436B3B
:103B700022F400421A434A6090F82410C90606D580
:103B800001688A68836B22F480521A438A6090F835
:103B90002410890606D501688A68C36B22F4005296
:103BA0001A438A6090F82410490611D501684A68C2
:103BB000036C22F480121A434A60016CB1F5801F35
:103BC00006D101684A68436C22F4C0021A434A6075
:103BD00090F82410090606D501684A68806C22F422
:103BE000002202434A607047F8B500250446C0F839
:103BF0008050FDF719FA0746206800686FF07E468E
:103C0000000708D53B4600224FF4001120460096DD
:103C100000F03EFA60B92068006840070AD53B46CC
:103C200000224FF480012046009600F031FA08B1DE
:103C30000320F8BD2020A067E067256684F8745053
:103C40000020F8BD10B5806A0021A0F85A10A0F835
:103C50005210FEF7DAF910BD70B5846AA06FE56FF7
:103C6000216889684FF00006090606D5212804D18D
:103C7000A4F85260204600F0AEF820688068400644
:103C800006D5222D04D1A4F85A60204600F07EF813
:103C9000D4F8800040F01000C4F880002046FEF701
:103CA000B4F970BD10B50146806A096809688906D3
:103CB0002DD40021A0F85A10016851E8002F22F4F9
:103CC000807241E80023002BF6D10168083151E8E9
:103CD000002F22F0010241E80023002BF5D10168FA
:103CE000083151E8002F22F0400241E80023002B68
:103CF000F5D12021C167016E012908D1016851E881
:103D0000002F22F0100241E80023002BF6D1016EB3
:103D1000012902D0FEF7C8FB10BDB0F85810FEF71D
:103D20002CF910BD10B5806A016E012902D0FEF792
:103D3000BCFB10BDB0F858104908FEF71EF910BDC5
:103D400010B50146806A09680968890616D4002101
:103D5000A0F852100168083151E8002F22F08002CB
:103D600041E80023002BF5D1016851E8002F42F013
:103D7000400241E80023002BF6D110BDFEF740FCC5
:103D800010BD10B5806AFEF73CFC10BD016851E81B
:103D9000002F22F4907241E80023002BF6D1016835
:103DA000083151E8002F22F0010241E80023002BE6
:103DB000F5D1016E012908D1016851E8002F22F0E8
:103DC000100241E80023002BF6D12021C167002119
:103DD000016641667047016851E8002F22F0C00279
:103DE00041E80023002BF6D12021816770470000B5
:103DF0002DE9F041044600682369A168E66919438A
:103E00006369002533431943704A0368704E334099
:103E10000B43036020684168E36821F44051194373
:103E200041602168A069914201D0236A18438B68E0
:103E300023F4306303438B60664B216866489942E4
:103E40000DD1D0F8880010F0030006D0012845D02D
:103E5000022833D0032830D142E001202EE05F4B0E
:103E600099420BD1D0F8880010F00C0026D004281D
:103E700024D0082830D00C281FD131E0584B99426B
:103E80000BD1D0F8880010F0300017D0102825D0C2
:103E9000202821D0302810D122E091420DD1D0F835
:103EA000880010F4406009D0B0F5806F16D0B0F5EE
:103EB000006F11D0B0F5406F12D01020494B002692
:103EC0004FF4004C91422ED160B1022813D0042847
:103ED0000BD0082872D10DE00220EFE70420EDE7B7
:103EE0000820EBE7FDF7FAFB01E0FDF71BFC030000
:103EF00001D164E06346626802EB420098425DD8FB
:103F0000B3EB023F5AD8190E1B0250081818714122
:103F10000023FCF7C9F9344AA0F5407191424DD80D
:103F20002168C8604BE0E1694FF6EF77614527D122
:103F3000092843D2DFE800F0050811420D42424251
:103F40001000FDF7CBFB01E0FDF7DAFB030004D125
:103F500035E0FDF7E7FBF9E763466068590001EBE0
:103F60005001B1FBF0F0A0F11001B94226D84FF694
:103F7000F0710140C0F3420001432068C1601EE0BF
:103F800009281BD2DFE800F00508111A0D1A1A1AC9
:103F90001000FDF7A3FB01E0FDF7B2FB030004D125
:103FA0000DE0FDF7BFFBF9E76346606803EB5001E6
:103FB000B1FBF0F0A0F11001B94205D90125666608
:103FC0002846A666BDE8F08180B2A9E700800040DF
:103FD000F369FFEF00380140001002400044004048
:103FE000004800400024F400FFFC0F0070B541655C
:103FF000A0F8582000250446C0F880502220E06731
:10400000206FD8B11F49C162216F1F481346086352
:10401000216F1E484863206F8563666D21683246B4
:104020002431206FFCF7F0FD40B11020C4F880006F
:1040300004F8745F2020A060012070BD84F87450E3
:10404000206940B1206850E8001F41F4807140E8C9
:104050000012002AF6D12068083050E8001F41F015
:10406000010140E80012002AF5D12068083050E82C
:10407000001F41F0400140E80012002AF5D1002065
:1040800070BD0000A53C0008253D0008593C000813
:104090002DE9F0471F4690460E4604464FF0000AB1
:1040A0004FF02009089D49E0681C47D0FCF7BCFF91
:1040B000C01BA8422AD84DB32068016849073DD5E6
:1040C000C069C043000539D421684FF4006008621C
:1040D000206850E8001F21F4D07140E80012002A47
:1040E000F6D12068083050E8001F21F0010140E8B7
:1040F0000012002AF5D1C4F87890C4F87C90C4F876
:10410000809084F874A00320BDE8F087206850E810
:10411000001F21F4D07140E80012002AF6D1206877
:10412000083050E8001F21F0010140E80012002A89
:10413000F5D1C4F87890C4F87C90E2E72068C069B3
:1041400036EA000004D000204045ADD00020DBE777
:104150000120F9E70B4810B50068C169C1F30011EF
:1041600059B1102101620748FDF709FF06480068B0
:1041700040680649C0F5A0700880BDE810400148BD
:10418000FDF744BF8C0C0020940D0020BC0A0020D9
:10419000FEE70000022901D0102070470249407854
:1041A000096888700120704740000020022908D16A
:1041B0004078411E062904D803490968C8700120C7
:1041C000704710207047000040000020042901D0F3
:1041D000102070470188827849BA0904C07841EA02
:1041E0000221014302480068C0F8F0100120704726
:1041F00040000020022901D01020704703490088A8
:10420000096840BAA1F8EE00012070474000002084
:10421000022901D01020704703490088096840BA7C
:10422000A1F8EC0001207047400000200FB4054BBE
:1042300010B503A9044A029800F03AF810BC5DF8E2
:1042400014FB000079450008340100200907090E1D
:10425000002804DB00F1E02080F80014704700F033
:104260000F0000F1E02080F8141D7047BFF34F8F5E
:1042700005480168054A01F4E06111430160BFF39C
:104280004F8F00BFFDE700000CED00E00400FA05D1
:1042900002E008C8121F08C1002AFAD1704770470F
:1042A000002001E001C1121F002AFBD1704700006D
:1042B0002DE9FF4F8DB09B460F460446002606E0D1
:1042C00025280BD05A460F999047641C761C2078FD
:1042D0000028F5D111B0304600F04AB90025A846B3
:1042E0000122984900E0054314F8013F203B02FAFF
:1042F00003F00842F7D120782E2817D114F8010FC7
:1043000045F004052A280ED06FF02F022078A0F186
:10431000300109290AD808EB880102EB410100EBC2
:104320000108641CF2E757F8048B641C20786C28A1
:104330000DD004DC4C2812D06A2811D104E0742876
:104340000DD07A280CD10AE045F4001507E0617819
:1043500045F48015814202D1641C05F58015641C6A
:104360002078692844D008DC0028B3D0582867D0CA
:1043700063280FD0642808D13AE0702865D07328EC
:1043800012D075285AD078285AD05A460F9990479B
:10439000761CD5E017F8040B8DF8000000208DF88E
:1043A0000100E946012003E057F8049B4FF0FF307D
:1043B00069074FF0000501D40AE06D1C45450DDA90
:1043C0008542FADB19F805100029F6D106E06D1CCC
:1043D0008542FCDB19F805100029F8D12E4404E0D1
:1043E00019F8010B5A460F9990476D1EF8D2A7E0B5
:1043F0000A200021CDE90801C5F3025002280CD0A3
:1044000001CFC117021E71F100020CDA0023D0EBBC
:10441000030063EB01012D2208E0FF1D27F00707D1
:10442000F7E80201EEE72A0504D52B228DF82820B3
:1044300001223CE0EA073AD02022F7E70A2000E018
:1044400010200021CDE9080107E01020002145F0EF
:104450000405CDE908014FF00808C5F30250022811
:1044600010D001CF00214FF0000A2A0720D5227872
:10447000702A0DD0DDE908C38CF0100C5CEA030C47
:104480000CD015E0FF1D27F00707F7E80201EAE767
:1044900040228DF828204FF0010A0CE050EA010379
:1044A00006D030238DF828308DF82920022292463C
:1044B0002278582A04D024A20DF120090B9209E099
:1044C00026A2F9E7DDE90823FBF7EEFE0B9B9B5CD8
:1044D00009F8013D50EA0102F4D1ADEB09002030AA
:1044E0000890680701D44FF001080899884503DD5A
:1044F0000898A8EB000000E000208046002506E0B8
:104500000AA85A46405D0F9990476D1C761C554588
:10451000F6DB04E030205A460F999047761CB8F13C
:104520000001A8F10108F5DC05E019F8010B5A4675
:104530000F999047761C0899481E08900029F4DCD2
:10454000641CC4E609280100303132333435363773
:1045500038396162636465660000000030313233CF
:10456000343536373839414243444546000000006F
:1045700030BCBDE8C08F000013B54FF6FF730122B9
:1045800069460248FDF792FF00981CBD100D0020FF
:104590000148FCF781BD0000AC0A0020FCF78AFD51
:1045A000FFF7C0F9FBF7BAFFFEF7B4FDFEF75EFDBB
:1045B000FEF742FEFEF78CFEFEF736FDFEF724FE08
:1045C000FFF7A0F800F0E2FAFEF76EFD00F0F0FA57
:1045D000FEE700002DE9F041764D4FF6FF7203260D
:1045E0002968888840BA02EA400468680A7802703C
:1045F000497841700021817029462A8A8989C91E1B
:104600000B2A7DD005DC5AB1082A47D0092A04D1EB
:104610008EE0102A75D0112A74D00220A8735AE0B7
:10462000102C06D0122C09D0162C15D0182C24D002
:1046300032E089B2C01CFEF7BBFF48E089B2C01C63
:10464000FEF7B6FFC01C87B2A889C01B81B268689C
:104650003844FEF7CDFF0EE089B2C01CFEF7A8FF7C
:10466000C01C87B2A889C01B81B268683844FEF7B5
:10467000BFFF384453E038442AE089B2C01CFEF73B
:1046800097FFC01C87B2A889C01B81B268683844F4
:10469000FEF7AEFF38440CE0AE731CE0022C12D0E3
:1046A000062C37D0082CF7D189B2C01CFEF7A0FF2A
:1046B000C01C87B2A889C01B81B268683844FEF765
:1046C00049FF38443DE089B2C01CFEF791FFC01C91
:1046D000A97B80B2F1B36868417841F080014170F4
:1046E000A97B81706E816989686800F0E3F9698946
:1046F0006A685054491C89B2000A5054491C02E0AF
:104700002EE034E04AE089B26981BDE8F04110460C
:1047100000F010BF89B2C01CFEF76AFFC01C87B250
:10472000A889C01B81B268683844FEF713FFA2E76E
:10473000042C10D0062CAFD189B2C01CFEF70AFFA2
:10474000C01C87B2A889C01B81B268683844FEF7D4
:104750001DFF90E729E089B2C01CFEF7FBFEB6E71B
:10476000022C99D189B2C01CFEF710FFAFE7022CD2
:104770000FD0042C90D189B2C01CFEF7CFFEC01C14
:1047800087B2A889C01B81B268683844FEF7D4FE9E
:1047900071E789B2C01CFEF7C1FE98E7022CCAD1AE
:1047A00089B2C01CFEF7C8FE91E769688C70688109
:1047B00099E700003801002070B5364D0024D5E996
:1047C00000102A89FBF7A4FD288A032608380A2846
:1047D00037D2DFE800F0053636102E303636192293
:1047E0002889082805D128680221001DFFF710FD3F
:1047F0001BE0AE7327E028890828FAD12868022137
:10480000001DFFF7F7FC10E028890828F1D128687F
:104810000221001DFFF7BEFC07E028890828E8D127
:1048200028680221001DFFF7C1FC04461028E0D0D3
:1048300004E0022402E0FEF7EDFE0324A87B28B387
:1048400001E00220A8736868417841F0800141705E
:10485000A97B817031466E8100F02CF969896A6804
:104860005054491C89B2000A5054491C6981698915
:10487000686800F05FFEE00701D0FEF7D1FEA007F8
:1048800007D56420FCF7F8F9FFF7F0FC2889688168
:10489000EDE770BD380100202DE9F0415E4F0024A6
:1048A00039683A8988888D7946BA7868FBF730FD8F
:1048B00030460326B5EB400F04D13889A0F1090139
:1048C000A94201D0BE737DE0B97B00297AD1398A33
:1048D00008390A2974D2DFE801F00530734B73738D
:1048E00073735369082D09D0062D18D00828E9D113
:1048F00038680221C01DFFF78BFC27E038680221D1
:10490000C01DFFF785FC0446386804210930FFF715
:104910005DFC40EA0405386802210D3025E0386866
:104920000221C01DFFF774FC0546386804210930D8
:10493000FFF74CFC40EA050409E0062D0CD0042DDD
:10494000C0D138680421C01DFFF740FC0446E006D2
:10495000B8D4B87B90B335E038680421C01DFFF7A8
:1049600035FC0546386802210B30FFF743FCE1E7D0
:10497000022DA7D138680221C01DFFF73BFCE5E7F7
:10498000042D07D0022D9DD138680221C01DFFF7EC
:1049900001FCDBE738680221C01DFFF7FBFB054681
:1049A000386802210930FFF7F5FBC3E7022D89D1F2
:1049B00038680221C01DFFF7F9FBC7E726E0FFE7D3
:1049C0000220B8737868417841F080014170B97B6A
:1049D00081707E817989786800F06CF879897A68CD
:1049E0005054491C89B2000A5054491C89B279813B
:1049F000104600F09FFDE00701D0FEF711FEA00772
:104A000007D56420FCF738F9FFF730FC06207881E1
:104A1000E0E7BDE8F08100003801002070B5234DCB
:104A20000024D5E900020168116004216981298A06
:104A3000A1F52A43BB3B02D00220A87310E02989CC
:104A4000001D891F89B2121DFDF7DEFD698908442A
:104A5000688117480078012800D10224A87B40B162
:104A60006868417841F080014170A97B8170032022
:104A700068816989686800F01DF869896A6850541E
:104A8000491C89B2000A5054491C89B269811046F8
:104A900000F050FDE00701D0FEF7C2FDA00704D5ED
:104AA0006420FCF7E9F8FFF7E1FB70BD3801002056
:104AB000540000200A4610B501460248FBF713FFD8
:104AC00080B210BD880A002010B50F4CD4E9001048
:104AD00009680160417841F08001417001218170D5
:104AE00003216181FFF7E6FF618962685054491C28
:104AF00089B2000A5054491C89B26181BDE8104056
:104B0000104600F017BD0000380100200C4A116863
:104B10004878D0734988032849BA118207D00628FB
:104B200007D0102807D0422807D0FFF7CDBFFFF7E6
:104B300051BDFFF741BEFFF7AFBEFFF76FBF0000EB
:104B40003801002010B5EFF3058111B16FF00504B5
:104B500003E0002408B100F03BFE204610BD10B574
:104B60004FF00001EFF305826AB948B1D0E90220A5
:104B70002AB1202807D3104600F07AFF02E010B9CE
:104B800000F068FF0146084610BD0000EFF3058005
:104B900010B16FF0050070470448016811B14FF083
:104BA000FF307047012101600020704704010020A0
:104BB00010B5EFF3058010B16FF0050010BD084887
:104BC0000168012902D04FF0FF3010BD054A0021D5
:104BD00082F8141D0221016000F0C0FE002010BD0B
:104BE000040100200BE000E02DE9FF410B464FF0EF
:104BF0000005EFF30581039549BB40B380261821DA
:104C000000244AB3176807B13C46976907B1394693
:104C10004F1E382F02D21779FF0703D0002004B0AF
:104C2000BDE8F081576907B1BE08D2F808C0BCF1F1
:104C3000000F0DD0D5685C2D18D312693AB137B189
:104C40008DE806103246214601F014FB03900DE07A
:104C5000D7685FB912694AB903AACDE90012B2B2A6
:104C6000214601F0D7FA012800D003950398D6E732
:104C70002DE9F041134E0F460446F5683068001DDB
:104C800000F068FC601C07D137B13168BDE8F04125
:104C90000D48091D00F0BABC30682C44AC42446099
:104CA000316805D2B06BBDE8F041091D00F096BC3B
:104CB000706B091D00F092FCB06A844200D2B462AD
:104CC000BDE8F081B4000020601300202DE9F04120
:104CD000054600F0A7FC2D4EB068401CB06030685F
:104CE0002B4F10B1706930B32BE03560B0680128EC
:104CF00027D1002404EB840007EB800000F060FC67
:104D0000641C382CF6D3234800F05AFC2148143098
:104D100000F056FC1F48283000F052FC1D483C3083
:104D200000F04EFC1B48503000F04AFC19487063FC
:104D30001430B06305E03068E96AC06A884200D880
:104D40003560706A401C70626864E86A3169884244
:104D500000D9306100EB800007EB8000291D00F0D6
:104D600055FC00F07FFC706900280CD03068E96ABF
:104D7000C06A884207D208494FF080500860BFF3EC
:104D80004F8FBFF36F8FBDE8F0810000B4000020AB
:104D9000B00E00201013002004ED00E038B500F044
:104DA00041FC104C2068C8B90F4800F009FC0E48BF
:104DB000143000F005FC0C48E060143020610A4B10
:104DC0000020F03B009003F1500210210A2000F077
:104DD000BFFF206010B105A100F0C6FCBDE838405F
:104DE00000F040BCF000002064140020546D7251AB
:104DF0000000000030B4026C0B46002A0BD0C168E2
:104E00001144C1608468A14201D30168C16030BC13
:104E10001846FBF77DBA30BC70472DE9F041856B31
:104E2000174604460026026C82B1C7B1E068FBF762
:104E30006FFAE168206C091AE1602268914202D29F
:104E4000A168081AE060022F16D017E02068A8B900
:104E5000A06801F0B5FA06460020A0600EE0606888
:104E6000FBF756FA216C606808446060A1688842CC
:104E700004D32068606001E005B16D1E6D1CA56360
:104E80003046BDE8F08110B5044690F8590058B19D
:104E900001280CD002280FD0502080F31188BFF3D6
:104EA0004F8FBFF36F8FFEE7206B00F0EFFB2046C4
:104EB000BDE8104000F0EABB10BD000010484FF400
:104EC000FA51420706D0C01D0D4920F00700411AD3
:104ED000C1F5FA510B4A00230144C2E90003083925
:104EE000183A21F0070111604B600B600B1AC0E902
:104EF000001393604FF00040536050617047000012
:104F0000441B002020010020134E144DA6F29C47A4
:104F10004FF08058DFF8489011E000F083FBF06814
:104F2000C468201D00F016FBA868401EA8606868D1
:104F3000401E686000F096FB2046FFF7A4FF6868FB
:104F40000028EAD138680128F9D9C9F80080BFF3F0
:104F50004F8FBFF36F8FF2E74C130020B400002097
:104F600004ED00E070B51D46049C49B12260C4E91F
:104F70000F010121204600F01FFF84F84C5070BD46
:104F80002460F4E72DE9F05F0E46DDE90B94174647
:104F9000834691009A460A9DA522206BFBF7CAF929
:104FA0006FF00301206B01EB8701084420F0070735
:104FB000780707D0502080F31188BFF34F8FBFF3DD
:104FC0006F8FFEE74FF0000866B100202218315CB9
:104FD00082F83410315C11B1401C1028F6D384F8EB
:104FE000438001E084F83480382D00D33725E56212
:104FF000C4E91358201D00F0EEFA04F1180000F087
:10500000EAFA2461C5F138006462A061C4F85480F2
:1050100084F8588052465946384600F069FA2060B4
:10502000B9F1000F01D0C9F8004000F000B830BC61
:10503000BDE8C09F30B5114900E011460A688242C0
:10504000FBD34B685C18844203D140681844486025
:10505000084643681C18944209D1084C183C24683F
:10506000A24209D052681A4442600A68126802607B
:10507000814200D0086030BD0460F9E720010020C3
:1050800070B5002441600B4D0061914206D8D11AE1
:105090008269914206D2011D286907E09A4203D233
:1050A000994201D3012403E0011DE86800F096FA5B
:1050B000204670BDF000002010B5044600F0B2FAA2
:1050C000A06B20B1002400F0CDFA204610BD0124D1
:1050D000F9E7000030B587B03C4D6EE0019800283C
:1050E00006DADDE90301029A90470198002864DBA3
:1050F000039C606910B1201D00F02CFA05A800F097
:10510000D7F8024601980A2857D2DFE800F00505D3
:10511000052D334A05052D3394F8280040F0010091
:1051200084F828000298A169034601442046FFF74D
:10513000A7FF68B3216A2046884794F828004007F3
:105140003BD5002000900298A1690023421819461F
:10515000204601F03BFAD8B9502080F31188BFF304
:105160004F8FBFF36F8FFEE714F8280F20F0010078
:10517000207022E094F8280040F0010084F8280014
:105180000298A06128B1811813462046FFF778FFE6
:1051900013E0502080F31188BFF34F8FBFF36F8F60
:1051A000FEE794F82800810703D4204600F06EFA49
:1051B00003E020F0010084F82800002201A92868FB
:1051C00000F052FF002889D107B030BDF000002068
:1051D0002DE9FC410F46054600F002FC01A800F055
:1051E00067F80446019818B101F060F9BDE8FC8148
:1051F000254EAFB130690068D0B30027291B3A466D
:10520000306800F0C3FA01F051F90028EED11F49CF
:105210004FF080500860BFF34F8FBFF36F8FE5E70B
:10522000A542EBD801F042F9F0682746C068C4688F
:10523000201D00F08FF994F82800410719D5A069C6
:105240002B4641193A462046FFF71AFFA8B1002025
:105250000346014600902A46204601F0B7F960B99E
:10526000502080F31188BFF34F8FBFF36F8FFEE79D
:1052700007E020F0010084F82800216A20468847D2
:10528000B4E70127BAE70000F000002004ED00E0D9
:105290000648416B096829B1416BC968C96849680A
:1052A000816270474FF0FF31FAE70000B400002040
:1052B00070B5054601F01AF8064E0446B0688442FF
:1052C00003D200F009F8012000E000202860204609
:1052D000B46070BDF0000020F8B5194E20E0C06841
:1052E000C4680568201D00F035F9216A204688470A
:1052F00094F82800400713D5A0692844A84206D98D
:1053000024616060211DF06800F068F908E0002069
:105310000346014600902A46204601F057F938B16D
:10532000F06801680029DAD13169C6E90310F8BDD7
:10533000502080F31188BFF34F8FBFF36F8FFEE7CC
:10534000F000002008484068401C4FF0500080F3F7
:10535000118804D0BFF34F8FBFF36F8FFEE7BFF309
:105360004F8FBFF36F8FFEE7280100200346002018
:1053700012B1994302D070470B42FCD00120704714
:10538000084CE068016839B1002139B10020FFF70D
:105390001FFFFFF79FFEF4E70121F6E7C0680068F2
:1053A000F5E70000F00000202DE9F041044600F090
:1053B00039F994F9455004F1240609E0606A48B1CE
:1053C000304601F03BF808B100F030FA6D1E6DB2C6
:1053D000002DF3DC4FF0FF3684F8456000F042F911
:1053E00000F020F994F9445004F1100709E0206915
:1053F00048B1384601F022F808B100F017FA6D1EE6
:105400006DB2002DF3DC84F84460BDE8F04100F09B
:1054100029B900002DE9F0410546002600F0E0FA28
:10542000324F386808B9FFF749FD786905424ED117
:10543000C5B3083568070ED005F00700C0F10800B5
:105440000544680707D0502080F31188BFF34F8FC1
:10545000BFF36F8FFEE72DB37868854237D82349B5
:1054600018310846046801E0214604466068A842F5
:1054700002D220680028F7D13868844227D00E680D
:105480002068086060680836411B10290FD9601930
:10549000420708D0502080F31188BFF34F8FBFF32D
:1054A0006F8FFEE713E041606560FFF7C3FD616841
:1054B0007868401A7860BA68904200D2B86078691B
:1054C00001430020C4E90001F868401CF86000F0C6
:1054D000EDFF700707D0502080F31188BFF34F8F86
:1054E000BFF36F8FFEE73046BDE8F0810801002072
:1054F00010B5031F4FF080741C601B1F21F00101C9
:105500001960191F044B0B6014390A60091F6FF0F2
:10551000020244380A6010BD4553000804480021C7
:105520004FF4A0720180416800F5E870FCF792BF6B
:10553000BC0A00200A4610B501460548FDF710F8E0
:10554000002803D0BDE81040FBF7E2B810BD000012
:105550008C0C0020D0E9013201699A60D0E9012366
:105560005A604A68824201D182684A600022026120
:105570000868401E08600868704700000449086811
:105580000A688069D26A0968C2F138028A61704784
:10559000B4000020034B036003F15C00086080202E
:1055A000106070478C140020044B036003F15C0012
:1055B00008604FF48070106070470000E81600200B
:1055C00000F108014FF0FF32C0E90112C160016132
:1055D00000210160704700210161704730B50C68FF
:1055E000621C02D000F1080202E0026904E01A46DF
:1055F00053681D68A542FAD953684B6099608A6068
:10560000516008610168491C016030BD42684A6010
:1056100093688B6093685960916008610168491CC8
:1056200001607047502080F31188BFF34F8FBFF3A4
:105630006F8F0A494868401C486001280CD108480F
:10564000006810F0FF0F07D0502080F31188BFF3DF
:105650004F8FBFF36F8FFEE77047000028010020D7
:1056600004ED00E00849486828B1401E486001D1B7
:1056700080F311887047502080F31188BFF34F8F5B
:10568000BFF36F8FFEE700002801002070B50028EF
:105690002AD0164DA0F1080460686969084207D154
:1056A000502080F31188BFF34F8FBFF36F8FFEE759
:1056B00022683AB1502080F31188BFF34F8FBFF3B7
:1056C0006F8FFEE78843606000F08AF96068696860
:1056D000084468602046FFF7ADFC2869401C28613B
:1056E000BDE8704000F0E2BE70BD0000080100207F
:1056F0004FF0E02000210161816105494FF47A7289
:105700000968B1FBF2F1491E41610721016170474F
:10571000B000002010B5FAF7A1FD114910280ED3F2
:1057200000F1E02090F8F0030A78904207D2502070
:1057300080F31188BFF34F8FBFF36F8FFEE70948E7
:105740000068896800F4E060884207D9502080F33F
:105750001188BFF34F8FBFF36F8FFEE710BD0000BE
:10576000280100200CED00E010B5074B002253F893
:1057700032401CB1521C082AF9D310BD43F8321034
:1057800003EBC201486010BD700E002070B51546D5
:105790000E460446FFF746FF94F944100020491CCA
:1057A00001D184F8440094F94510491C01D184F8D2
:1057B0004500FFF757FFA06B28B92A46314604F190
:1057C000240000F051F82046BDE87040FFF7ECBD22
:1057D00010B5020014D00F48006B38B1502080F390
:1057E0001188BFF34F8FBFF36F8FFEE700F0F8F81B
:1057F00000211046FFF73CFA00F058FE002807D1C0
:1058000005494FF080500860BFF34F8FBFF36F8F93
:1058100010BD0000B400002004ED00E002490A6A57
:105820000260C96841607047B4000020014901204E
:10583000C8617047B400002010B50C4650B109494A
:1058400009681831FFF7CAFE2046BDE81040012163
:10585000FFF70EBA502080F31188BFF34F8FBFF3CC
:105860006F8FFEE7B400002070B514460D4668B196
:105870000A4909681831FFF7C9FE0CB14FF0FF352E
:1058800021462846BDE87040FFF7F2B9502080F36A
:105890001188BFF34F8FBFF36F8FFEE7B400002076
:1058A00010B5144680B1104B1A6BAAB11A6841F0BA
:1058B0000041916119681831FFF7A8FE2046BDE844
:1058C00010400121FFF7D4B9502080F31188BFF3B5
:1058D0004F8FBFF36F8FFEE7502080F31188BFF327
:1058E0004F8FBFF36F8FFEE7B400002070B5194DE6
:1058F0002A6BF2B141F000410160C4680CB3FFF7BC
:1059000029FE201DFFF726FEE06A2969884200D99A
:10591000286100EB8001104800EB8100211DFFF79A
:1059200075FEE06A2968C96A884201D90120E861E8
:1059300070BD502080F31188BFF34F8FBFF36F8F7E
:10594000FEE7502080F31188BFF34F8FBFF36F8FB6
:10595000FEE70000B4000020B00E002030B587B094
:105960000025039505AA04A903A80495FFF712FED4
:10597000DDE903010095CDE90110002314A11648CB
:10598000059A00F077FC154CE06218B100F0EEFDCE
:10599000012809D0401C19D1502080F31188BFF391
:1059A0004F8FBFF36F8FFEE7502080F31188BFF356
:1059B0004F8FBFF36F8F4FF0FF30A0620120606107
:1059C000E56007B0BDE8304000F032B907B030BD47
:1059D00049444C4500000000094F0008B400002075
:1059E0000248016B491C016370470000B4000020AD
:1059F000164B10B5186B10B10120D86110BD0020F6
:105A0000D8611869124901E0B8B1401E00EB80026C
:105A100051F82220002AF7D000EB800201EB82012E
:105A200001F108044A6852684A60A24201D15268F2
:105A30004A60D1681960186110BD502080F3118848
:105A4000BFF34F8FBFF36F8FFEE70000B40000205D
:105A5000B00E002070B52020FFF7DCFC040005D05C
:105A60000025201D2560FFF7ABFD2577204670BD82
:105A700038B558B120210446002000912060201D37
:105A8000FFF79EFD01202077204638BD502080F38F
:105A90001188BFF34F8FBFF36F8FFEE72DE9F04101
:105AA0000025884604000AD05FEA18600FD0502015
:105AB00080F31188BFF34F8FBFF36F8FFEE7502045
:105AC00080F31188BFF34F8FBFF36F8FFEE7261D62
:105AD00004F10C07FFF784FF2168F06841EA080130
:105AE000216017E0D0E9001601F07F4253012368DE
:105AF00021F07F4102D40B4203D10AE031EA0303D3
:105B000007D1D20100D50D43216841F00071FFF7A4
:105B1000EDFE3046B842E5D12068A843206000F091
:105B2000C5FC2068BDE8F0812DE9F0479A46089F42
:105B300091460D4604004FF0000609D0280E0FD004
:105B4000502080F31188BFF34F8FBFF36F8FFEE7B4
:105B5000502080F31188BFF34F8FBFF36F8FFEE7A4
:105B60001DB100F0B5FB40B110E0502080F311886A
:105B7000BFF34F8FBFF36F8FFEE73FB1502080F32D
:105B80001188BFF34F8FBFF36F8FFEE7FFF728FF3A
:105B9000D4F80080524629464046FFF7E7FB40B163
:105BA00000274646B9F1000F15D02068A8432060B1
:105BB00011E0AFB1B9F1000F01D04FF08076BAF12A
:105BC000000F01D046F0806645EA06013A46201DE6
:105BD000FFF766FE002600F069FC1FB310B109E074
:105BE0004646F8E711494FF080500860BFF34F8FE9
:105BF000BFF36F8FFFF7C2FC0646800110D4FFF79A
:105C000011FD2668524629463046FFF7AFFB28B102
:105C1000B9F1000F02D02068A8432060FFF722FDF1
:105C200026F07F463046BDE8F087000004ED00E036
:105C30001CB537480168374A914207D1502080F39C
:105C40001188BFF34F8FBFF36F8FFEE700683149B4
:105C5000491E884207D1502080F31188BFF34F8F2F
:105C6000BFF36F8FFEE72C4908780190FF20087082
:105C700008788DF800009DF800009DF8002000F0E5
:105C8000F000904207D0502080F31188BFF34F8F6F
:105C9000BFF36F8FFEE79DF80000204C00F050002E
:105CA00020700720A06006E0401EA0609DF8000064
:105CB00040008DF800009DF800000006A068F3D4B5
:105CC000032807D0502080F31188BFF34F8FBFF314
:105CD0006F8FFEE74FF44070A060019808700C4889
:105CE0002030016841F470010160016841F07041A9
:105CF0000160FFF7FDFC00206060FAF777FA0848C2
:105D0000016841F040410160FAF75CFA00201CBDD7
:105D100000ED00E071C20F4100E400E02801002026
:105D200034EF00E010B5502080F31188BFF34F8F9F
:105D3000BFF36F8F00F0E0FA18B104494FF08050C4
:105D40000860002080F3118810BD000004ED00E021
:105D500038B5049D18B153B1CAB181B120E05020CB
:105D600080F31188BFF34F8FBFF36F8FFEE7502092
:105D700080F31188BFF34F8FBFF36F8FFEE7502082
:105D800080F31188BFF34F8FBFF36F8FFEE739B1F8
:105D9000502080F31188BFF34F8FBFF36F8FFEE762
:105DA00050241C46012384F846302B460094FFF70C
:105DB000D9F8204638BD000070B50D46040025D046
:105DC000FFF730FCD4E90F20216802FB0011A1602D
:105DD0000021A163216861600A46D4E90F01401ED9
:105DE00000FB0121E16021464FF0FF3001F8440F34
:105DF000487004F110008DB1FFF7E2FB04F12400BC
:105E0000FFF7DEFBFFF72EFC012070BD502080F372
:105E10001188BFF34F8FBFF36F8FFEE72169002911
:105E2000F0D000F00BFB0028ECD004494FF080507C
:105E30000860BFF34F8FBFF36F8FE3E704ED00E01F
:105E40002DE9FF4F83B01F468B4604004FF000063C
:105E500003D0BBF1000F08D011E0502080F311886F
:105E6000BFF34F8FBFF36F8FFEE7206C38B1502028
:105E700080F31188BFF34F8FBFF36F8FFEE7022FC0
:105E80000AD1E06B012807D0502080F31188BFF3BE
:105E90004F8FBFF36F8FFEE700F01AFADFF8009123
:105EA0004FF0000A4FF0805848B9059838B150209B
:105EB00080F31188BFF34F8FBFF36F8FFEE7FFF7BB
:105EC000B1FBA06BE16B884205D3022F03D005988C
:105ED000C8B1DEB11EE03A4659462046FEF79DFFA6
:105EE000616A19B104F1240000F0A8FA28B1C9F8D8
:105EF0000080BFF34F8FBFF36F8FFFF7B3FB01201D
:105F000007B000F04FB8FFF7ADFB21E06846FFF7A0
:105F100085FC0126FFF7A6FBFFF762FDFFF782FB7A
:105F200094F94400401C01D184F844A094F9450040
:105F3000401C01D184F845A0FFF794FB05A96846F1
:105F400000F02EF930B12046FFF72EFA00F0AEFA3D
:105F50000020D5E7FFF766FBA06BE16B884201D11B
:105F6000012500E00025FFF77DFB95B104F110004D
:105F70000599FFF761FC2046FFF716FA00F096FA44
:105F800000289CD1C9F80080BFF34F8FBFF36F8FFB
:105F900095E72046FFF708FA00F088FA8FE700003F
:105FA00004ED00E030BCBDE8C08F2DE9F0471F468E
:105FB00090468946040003D0B9F1000F08D011E0E3
:105FC000502080F31188BFF34F8FBFF36F8FFEE730
:105FD000206C38B1502080F31188BFF34F8FBFF38E
:105FE0006F8FFEE7022F0AD1E06B012807D0502007
:105FF00080F31188BFF34F8FBFF36F8FFEE7FFF77A
:1060000089FB5020EFF3118680F31188BFF34F8F87
:10601000BFF36F8FA06BE16B884206D3022F04D0D1
:10602000002086F31188BDE8F08794F94550A06BF5
:106030003A4649462046FEF7F0FE681C04D06D1C27
:1060400084F845500120ECE7606A0028FAD004F19A
:10605000240000F0F3F90028F4D0B8F1000FF1D0DB
:106060000121C8F80010EDE72DE9F74783B08A4613
:1060700004004FF0000603D0BAF1000F08D011E081
:10608000502080F31188BFF34F8FBFF36F8FFEE76F
:10609000206C38B1502080F31188BFF34F8FBFF3CD
:1060A0006F8FFEE700F014F9DFF8F09000274FF053
:1060B000805848B9059838B1502080F31188BFF353
:1060C0004F8FBFF36F8FFEE7FFF7ACFAA56BC5B13B
:1060D00051462046FEF78EFE6D1EA563206950B125
:1060E00004F1100000F0AAF928B1C9F80080BFF34C
:1060F0004F8FBFF36F8FFFF7B5FA012006B0BDE8F1
:10610000F087059808B11EB106E0FFF7ABFA27E06B
:106110006846FFF783FB0126FFF7A4FAFFF760FC50
:10612000FFF780FA94F94400401C01D184F84470D0
:1061300094F94500401C01D184F84570FFF792FAAC
:1061400005A9684600F02CF8002820460AD0FFF781
:106150002BF900F0ABF92046FEF7AEFF0028B3D0D4
:106160000020CBE7FEF7A8FF90B104F124000599C9
:10617000FFF762FB2046FFF717F900F097F90028B8
:10618000A2D1C9F80080BFF34F8FBFF36F8F9BE799
:106190002046FFF709F900F089F995E704ED00E0E2
:1061A0002DE9F0410C46050011D0C4B1FFF73AFAD1
:1061B000174EF1686B682268C81A571C17D02F68F1
:1061C000366AB74219D08B4217D8012410E050200C
:1061D00080F31188BFF34F8FBFF36F8FFEE750201E
:1061E00080F31188BFF34F8FBFF36F8FFEE700245A
:1061F000FFF738FA2046BDE8F081824205D9101A2F
:1062000020602846FFF70AFBF1E700202060DCE76A
:10621000B40000202DE9FF5F8346DDE90E87994633
:1062200016468A469000FFF7F5F805001CD05C2062
:10623000FFF7F0F8040014D00020256384F859001B
:10624000CDE90240CDE900874B46324651465846DB
:10625000FEF798FE2046FEF739FD012004B000F05D
:1062600006B82846FFF712FA4FF0FF30F6E730BCC9
:10627000BDE8C09FF0B585B00546DDE90B040A9E78
:10628000A8B1E4B15C2700972063022084F859008C
:106290000020CDE9024004AF2846CDE90067FEF7B3
:1062A00071FE2046FEF712FD049805B0F0BD5020A7
:1062B00080F31188BFF34F8FBFF36F8FFEE750203D
:1062C00080F31188BFF34F8FBFF36F8FFEE700009D
:1062D0000548416919B1006B18B1002070470120D1
:1062E0007047022070470000B40000200148C068D9
:1062F00070470000B40000202DE9F0412E4F002629
:10630000386B28B1B869401CB8613046BDE8F081EF
:10631000FD686D1CFD6013D1786B006838B15020AA
:1063200080F31188BFF34F8FBFF36F8FFEE7786B59
:10633000B96B7963B863386A401C3862FEF7A8FF0E
:10634000B86ADFF87880854209D3786B0068A0B11D
:10635000786BC068C4686068854211D2B8623868DA
:10636000C06A00EB800158F82100012800D90126FD
:10637000F8690028C9D00126C7E74FF0FF30EDE7E4
:10638000201DFFF7E7F8A06A18B104F11800FFF725
:10639000E1F8E06A3969884200D9386100EB800190
:1063A00008EB8100211DFFF731F9E06A3968C96AFD
:1063B0008842CAD30126C8E7B4000020B00E0020EE
:1063C00070B504004FF000002BD01A4D29688C42A4
:1063D00007D0502080F31188BFF34F8FBFF36F8F2A
:1063E000FEE7216DF1B1491E2165E36CE26A9A4234
:1063F00017D0002915D1201DFFF7ACF8E06CE06242
:10640000C0F13800A061E06A2969884200D928619A
:10641000094900EB800001EB8000211DFFF7F6F831
:10642000012070BD502080F31188BFF34F8FBFF360
:106430006F8FFEE7B4000020B00E002070B5C0687A
:10644000C46854B104F118000646FFF783F8144DF0
:10645000286B50B13146134815E0502080F3118865
:10646000BFF34F8FBFF36F8FFEE7201DFFF772F86A
:10647000E06A2969884200D928610B4900EB800055
:1064800001EB8000211DFFF7C1F8E06A2968C96AA5
:10649000884202D90120E86170BD002070BD000073
:1064A000B400002038130020B00E00202DE9F04782
:1064B0002B4D00242746286B38B1FFF7B3F8286B23
:1064C000401E2863286B40B145E0502080F31188BE
:1064D000BFF34F8FBFF36F8FFEE7A86821490126F6
:1064E000C8B3A1F591698846D8F80010E1B1D8F891
:1064F0000C00C46804F11800FFF72CF8201DFFF70A
:1065000029F8E06A2969884200D9286100EB8001F6
:1065100009EB8100211DFFF779F8E06A2968C96A53
:106520008842E1D3EE61DFE70CB1FEF7B1FEAC6962
:106530003CB1FFF7E1FE00B1EE61641EF9D100202D
:10654000A861E86938B10849012738070860BFF336
:106550004F8FBFF36F8FFFF785F83846BDE8F087A0
:10656000B40000203813002004ED00E010B586B020
:10657000FEF714FC114C2068B8B100200390049081
:1065800005AA04A903A8FFF70FF8DDE903210220FB
:106590008DE8070000230AA10B48059AFFF76AFE61
:1065A000606010B106B0012010BD502080F311884A
:1065B000BFF34F8FBFF36F8FFEE70000F0000020A6
:1065C000546D722053766300815300082DE9FF411A
:1065D0001F4603000A9E4FF0000015D0134D2C6893
:1065E000002C0ED08DE80E00062917DAFFF770FE9A
:1065F00002284FF000030FD0002269462868FFF7F9
:106600001FFC04B0BDE8F081502080F31188BFF377
:106610004F8FBFF36F8FFEE73246EEE700233A4617
:1066200069462046FFF7C1FCEBE70000F0000020C0
:1066300010670008000000000000000000000000DB
:106640000000000000020000180000000000000030
:1066500000000000046700080000000000000000C7
:106660000000000000000000000200001800000010
:106670000000000000000000F466000800000000B8
:106680000000000000000000000000000002000008
:106690001000000000000000000000001C6700085F
:1066A00000000000680A0020200000000000000038
:1066B000000000000102030406070809A08601008B
:1066C000400D0300801A060000350C0040420F0008
:1066D00080841E0000093D0000127A000024F400AE
:1066E00000366E010048E801006CDC02000000008A
:1066F000010203045761746368646F675461736BCC
:10670000000000004D6F646275735461736B00008C
:1067100064656661756C745461736B007461736B4E
:106720004576656E74000000486700080000002090
:1067300038010000D40300086C670008380100200D
:10674000503D0000A0420008024080865001002019
:10675000014201053102FE3401420102181002110A
:0C67600001037A093D95AAAAAAAA00002C
:040000050800018D61
:00000001FF
